S1048000007B
S123C000C787C769C790C7C4C76FC777C77FC7D2C7EAC7E2C7F2C844C83AC82EC833C84D42
S123C020C865C8B3C875C885C895C93BC95BC967C97BC78DCA5EC991C9A6C99BCABACAC614
S123C040CAD1C9C3C9AFC9CDC9D7C9E7CA28CA54CA63CA7FCA8ECA9DCA34CA44CA19C9FF5B
S123C060CAE6CAEACAF0CB01CB14CB07CB4ACB1CCB5ACBBDCBD2CBE0CBF2CB95CB9FCB7866
S123C080CBA8D7CED77AD7A4D7BCD7E1D7F4D806D811D829D84ED85ED7FFD879D88DD89882
S123C0A0D86ED8A3D8AED8B9D8CBD8D9D8E7D789D90FD934D91FD8F5DD46DE24DE28DE6D01
S111C0C0DAE2CBABCBB4DABBDAF1DB02000080
S123C500FCFF0227358E00FFBDE1411AB3FF022608CC0000FDFF022021BDDBD6CEC52DBD60
S123C520DD35B67F0084C088C027F720134D454D4F5259204641554C54008EFEFF7F003C18
S123C5408D392016B67F0084038103260D8E00FF0FBDE141FDFF027EE0DDB67F00848088F3
S123C5608027037EC712B680004A26F7CC8001CEC300ED008600A7097EC712CE002A4FA7D3
S123C58000088C003926F8CE1000860AB77F00970E86FF9722972397249725CC07C0DD265E
S123C5A01C39801D282086B0A72B860CA72D86079739BDDBD6CC0000DD0CDD12DD148608E1
S123C5C0970BCCC110DD16DD18DD1A8620B7C6F8CEC300C6208640A7098FC300108F5A26C0
S123C5E0F6CEC300DF08CCC200ED00CCFE00ED04C30001ED02830100ED06860AA708862084
S123C600A709EF0CEF0EDC0CC30001DD0CED0ABDDB02CEC639A6002706BDDBA80820F6CE7C
S123C62010001C200118CE3000180926FC1D20011D0008CC0000DD2639496E74657261631F
S123C6407469766520432020205620322E383120392F32382F39330A008D6B8D7481612585
S123C660F881732604863E2068368D513C18388D4C328172270D8177270F81632711816255
S123C680271B39A6008D4A2010188FE700200A188FA400A700EA00E700863E2034188F37FD
S123C6A03C32331B331B97015D270C8D19A7009B019701085A26F496018D1620DC8D073647
S123C6C08D0416328F39B6102E842027F9B6102F39F6102EC48027F9B7102F39DE08A60874
S123C6E0970A1AEE00EE0218E600F7C6F11808FCC000FDC6F6BDFFFF20ED8620B7C6F8DC9D
S123C700088FED021AEF00A60981402604EE0CDF0839963C260CCE10001F2E2005BDC659A2
S123C72020F0120B02ECDE08EE0EDF088CC3002607DC1EC30001DD1EA609810026D4BDC62F
S123C740DC810027CD814027C9812027048602200286048D0220BB9701940B910126013940
S123C76096019A0B970B7EC6D1EC02A300201CEC02A400E4012014EC02AA00EA01200CECAF
S123C78002A800E8012004EC00E302ED020808398D26A601E6033DDD00A600E6033DDB00D1
S123C7A0D700EC013DDB00D7007D000727064F5F930020D7DC0020D37F00078D6308088DF7
S123C7C05F090939BDC7B8EC023CEE0002DF003820D7EC00A3022705CC000020AECC000123
S123C7E020A9EC02A3002EF520EEEC02A3002DED20E63CEC002B1C260438080839373686EC
S123C80005B7C807EC02380027030926FA380808ED00394F5FA30037368604B7C80720E4D0
S123C8206D002A094F5FA300ED007300073963006301394F5FA300ED0039EC002705CC0008
S123C84001ED0039EC0027F64F5FED0039EC02E306DD00E601E905A600A904ED04DC00ED3A
S123C86006C6043A39EC06A302DD00E605E201A604A20020E6EC06A302E605E201A604A22C
S123C880002D1E2025EC02A306E601E205A600A2042D0E2015EC06A302260FEC04A300265E
S123C8A009C6063ACC0001ED0039C6063ACC0000ED00397F0007BDC9513CC6043ABDC95106
S123C8C0CE0000DF0038A603E6073DDD02A603E6063DD301DD01960089009700A602E607EE
S123C8E03DD301DD01960089009700A603E6053DD300DD00A602E6063DD300DD00A601E600
S123C900073DD300DD00EC033DDB00D700A602E6053DDB00D700A601E6063DDB00D700A697
S123C92000E6073DDB00D700C6043ADC02ED02DC00ED007D000727028D0139CC0000A30298
S123C940DD00C600E2018600A200ED00DC00ED02396D002A058DE47300073918EC00180850
S123C96018080909ED003918EC020909ED0018EC00180818081808180820E718E600183A7B
S123C98018A60009A70018095A26F518E600183A393CCDEE00E600384F20C38FCDEE00EE87
S123C9A0028F0909ED008FCDEE00EE008F20AF18E6003C3AEC00DD00EC02380909ED00DC0F
S123C9C000209D18E6003C3AEC003820933CA601CDEE00A70020083CEC00CDEE00ED0018F6
S123C9E0083818080808393CEC00DD00EC02CDEE00ED02DC00ED0038C6043A57183A39EC1A
S123CA0000DD00EC02D70718E6003C3AD607ED02DC00ED0038080820C9EC00D70118E6006D
S123CA203C3AD601ED0020B9A6013CEE02273FA70038202AA601B7CA403CEE0227301C0076
S123CA40FF38201AA601B7CA503CEE0227201D00FF38200AEC003CEE022713ED0038080871
S123CA60080839EC00DD00EC023CEE0426063886057EDE79ED02DC00ED0038080820DFECD5
S123CA80003CEE0227E8E70038ED02080839EC003CEE0227D9ED0038ED02080839EC00DDC2
S123CAA000EC023CEE0427C6ED02DC00ED0038EC02ED04DC00ED020808393CEE0027AFE6A0
S123CAC0004F38ED00393CEE0027A3EC0038ED00393CEE002798EC00DD00EC02380909ED90
S123CAE002DC00ED003918EE00391AEE00080839EC00260618EE00080839180818080808E7
S123CB0039EC0026EF20F3EC0027EFCC0001ED0018EE0039EC0026E218EE0039EC00DD00CD
S123CB2018EC00DF04D3048F1AEE002705DC00ED0039DE088640A7098621B7C6F8EC0C1AE4
S123CB40EE0E8FCDEF0C1AEF0E3918EC00DF00D3008F1AEE0027DB080839EC00DD00EC02DF
S123CB60DD0218EC00DF04D3048F1AEE0227C3DC00ED00DC02ED0239DF00DE08DC00A30678
S123CB80CDA300250718081808DE00391809DE0086047EDE798F18E3008F18081808393C72
S123CBA0323318E3007EC95EEE0039EC00DD3A0808180839DC3A0909ED00180839EC003C43
S123CBC0EE021AA300382427E302C30002ED02080839EC003CEE021AA3003824120520E8EF
S123CBE0EC003CEE021AA300382404050520D97EDE73EC003CEE021AA3003824F218A60049
S123CC0018083D20C33CBDD6EACE00003CDF3DDF3F7F00411830CDEE06A600BDCD5D252830
S123CC20812D260B73004108A600BDCD5D2519812E260B08A600BDCD5D24037ECCCB313177
S123CC40BDD6F438860F0D39A600BDCD5D2477BDCCDC0824F37C003DA60008BDCD5D25F522
S123CC60812E260AA600BDCD5D24030820F681452707816527037ECD1F08A600BDCD5D25D7
S123CC8015812D2706812B270520B318630008A600BDCD5D24A8803018A70108A600BDCD71
S123CCA05D241418E601585818EB015880301B18A701088126228718A601186D002A01403E
S123CCC09B3D973D2059812E26A408A600BDCD5D249C8D0808258D7A003D20EF963E97439A
S123CCE0DC3FDD440579003E252C0579003E2526D34436963E9943973E32251A0579003EE1
S123CD00DD3F2512E600C0304FD33FDD3F963E89002503973E39DC44DD3F9643973E39CDE6
S123CD20EF06CE003DBDCD88272C963D18A7018696973DBDCD69186D01271B2A0BCECD93E9
S123CD40BDD71D1860012006CECD97BDD71DBDCDA7186A0126F83131BDD6F438398130259A
S123CD6006813922020D390C39CE003D8D1A27147D003E2B0FDC3F7A003D270A0579003E9F
S123CD802AF5DD3F0C390D393736EC002602EC023233393DCCCCCD41200000BDD043BDD656
S123CDA0EABDCF12BDD6F47D003D27057D0042260ACC00009741DD3DDD3F3996419846972C
S123CDC041963D9B422A0924168606CEFFFF2009250D8607CE0000DF40DF3DDF3F0D398BB9
S123CDE082973DCE00003C3C30BDCE206D002B0B69036902690169007A003D6D032A13A661
S123CE00024CA702260CC601E3002404467C003DED0038DF3E329740317D003D27B45F396B
S123CE209645D6403DA7019644D6403DE300ED009645D63F3DE300A70324026C026F006FEF
S123CE40019643D6403DE302ED029644D63F3DE302ED0224026C019645D63E3DE302ED023A
S123CE6024026C019643D63F3DE301ED0124026C009644D63E3DE301ED0124026C00964324
S123CE80D63E3DE300ED0039BDD6EACED416BDD71D7D00412703730046BDCF44BDD6F44F07
S123CEA0D63DC17F24035F201B53C3FF902F178FDC3E2001040926FC7D00412A074353C32E
S123CEC000012A020C3986090D39CC0000DD004FD63DC17F24035F203353C3FFA02F2F8F41
S123CEE096405FDD00DC3E2007047600007600010926F67D00412A1473000073000143534C
S123CF00DE0008DF002605C300012A020C3986090D39BDD37ECE0045964280972A1BC603F5
S123CF208B082A096F00095A26F66F0039C6804A2B035720FAE400E7008D028D0796468810
S123CF40FF974639963D260EDC42DD3DDC44DD3F964697415F397D004227F9D641D846904D
S123CF60422510811822ED183C36CE004318CE003E201740811822D0183C369642973D9601
S123CF80469741CE003E18CE004317363636A8003617A8013617A8023630A606E706168453
S123CFA0074CC4185454543AE6034A27095666026601660020F45618A602A900974018A6B2
S123CFC001A901973F18A600A902973E30A6062B15245A76003E76003F7600407C003D26F6
S123CFE04CCCCDC92053251B73004170004024087C003F26037C003E70003F24037C003E0E
S123D00070003E7D003E2B252613963D80082326973DDC3F27207F0040DD3E20E67A003DA9
S123D020271478004079003F79003E2AF01AEE07C6093A355F39CCCDD21AEE07ED07C60750
S123D0403A3539CE0042BDCD88260486080D39CE003DBDCD8826020C39BDD6EA9646984148
S123D0609741CE00003C3C3C86183630DC3E1A934326049640914524107C004226198606B1
S123D0800D38383831BDD6F439DC3F9344DD3F963E9243973E6A00740043760044760045C4
S123D0A0963DD642501B2B062506860720D325CE8B7F973DDC3EED049640A706DC3F9344E9
S123D0C0DD3F963E9243973E2A08EC04DD3EA606974069036902690178004079003F7900C8
S123D0E03E6A0026CF630163026303DC3F9344963E9243EC0224030C2003C30001DD3FA6FB
S123D100018900973E241176003E76003F7600407C003D26037ED07E0C7ED0813CCE003D88
S123D120BDCD88260738CC3000ED0039DE3D3CDE3F3C964136BDD6EACE00003C3C3C18304E
S123D140CDEE0F86207D004127057F0041862DA70008CDEF00CED286BDD71DBDD28A2E195C
S123D160CED282BDD71DBDD28A2E16186A02CECD97BDD71DBDCDA720DC186C02CECD932013
S123D180F0CED416BDD71DBDCF44D63DC07F50CB17200A74003E76003F7600405A26F4869D
S123D1A00118A70318A6028B082B0A810824064A18A7038602800218A702186D032E158645
S123D1C02ECDEE00A70008186D0327058630A70008CDEF00CED26D860718A705186F04DC19
S123D1E03FA301DD3F963EA200973E2505186C0420EDDC3FE301DD3F963EA900973E18A6F7
S123D200048B303CCDEE00A70008186A032605862EA70008CDEF0038080808186A0526BC1D
S123D220CDEE0009A600813027F90818E602272A8645A70008862BA7005D2A0550862DA74E
S123D2400008CDEF004FCE000A02378FCB30CDEE00E7000833CB30E700086F00383838BD81
S123D260D6F432974138DF3F38DF3D38390F42400186A00027100003E800006400000A0073
S123D2800001497423FE4B18967F96462A12D6412A0EDC421A933D2617DC441A933F20104B
S123D2A09141260CDC3D1A93422605DC3F1A93440784F424028A080639CE008EC30000266C
S123D2C0057ECDD209052AFCDD3E7F00408F9741D73D5F394D2AE24353C30001CEFF8E20D9
S123D2E0DBCE009EC30000261118DE0026037ECDD20978000179000059492AF5DD3E960040
S123D30097408F9741D73D5F394D2AD57300007300014353DE0008DF002603C30001CEFFD7
S123D3209E20C1CE003DBDCD882601397D00412A04860A0D39BDD6EA860436DE3F3CDE3D7A
S123D3403C18308D399642807E4C2A03442003448B7E9742BDD043BDCF447A003D8D1F1888
S123D360EC00DD3D18EC02DD3F186A0426E6DC42DD3DDC44DD3F383831BDD6F45F39DC3DA2
S123D380DD42DC3FDD449641974639BDD6EACED4E5BDD71DBDD043BDD6F4DC3D1A8385B347
S123D3A02B0B7D004126037ECDC97ECDD2BDD6EA9641367F0041BDCF12DC4227068086548E
S123D3C04C26FC5C37CED3FABDD6AACED3F6BDD71D2003BDCDA7306A0026F832324D2A0C35
S123D3E0BDD37ECED63EBDD704BDD043BDD6F45F39BDD6EA20EA402DF8543638EF1D37D0F1
S123D4000D0139500D013AB60B613C0888893D2AAAAB3E2AAAAB3F0000003F8000003F807C
S123D4200000FFBDD43FBDCDA77ED39A8D11BDD6EACED4E5BDD71DBDCDA7BDD6F45F3996C4
S123D440412704860C0D39963D27F8BDD6EA3C3C30BDD7354FD63DC07F2A0143BDD2D4CE64
S123D460D4E1BDD71DBDCDA730BDD71DBDD735867F97423C3C30BDD743CED63EBDD704BDD3
S123D480CF4430BDD71DBDD735CED4DDBDD704BDCF4430BDD71DBDD04330BDD735BDD37E2C
S123D4A0BDCDA7CED4C0BDD6AA30BDD71DBDCDA7383830BDD71DBDCF443838BDD6F45F39D6
S123D4C03E1D89D93E3A2E8C3E638E393E9249253ECCCCCD3F2AAAAB40000000FFBF8000D4
S123D4E0003F3172183EDE5BD9860E0D39860D0D39BDD6EA9641367F0041CED63EBDD71D4E
S123D500BDD28A2F07BDD3F186FF20014F363C3C30BDD735BDD37EBDCDA7CED548BDD6AA34
S123D52030BDD71DBDCDA73838324D270CCED544BDD71D730041BDCF44BDD694329741BDA9
S123D540D6F45F393FC90FDBBCE2DD1B3D70F0F1BD8888893D9D89D9BDBA2E8C3DE38E39A5
S123D560BE1249253E4CCCCDBEAAAAAB3F800000FFBDD6EA4F2005BDD6EA86F036CED65CB1
S123D580BDD71D2003BDCF44964126F92003BDCF39BDD28A2EF88D61240930A6002B04881E
S123D5A00FA7008D54240930A6002A04880FA7008D47240730A60088F0A700CED6A2BDD793
S123D5C01DBDCDA7BDD37EBDCDA73C3C30BDD743A6042A05CED6432003CED62EBDD6AA3019
S123D5E0A6044724037300414D2B06BDD71DBDCDA7383831BDD6F45F397A0042BDD28A2E38
S123D600020C397C0042730041BDCF447A00420D39BDCF12DC3DDE42DD42DF3DDC3FDE442C
S123D620DD44DF3F9641D6469746D7415F393638EF1DB9500D013C088889BE2AAAAB3F8045
S123D6400000FF37D00D01BAB60B613D2AAAABBF0000003F800000FF40490FDB43B4000033
S123D660BDD6EABDD37EBDD577BDD614BDD571BDD0432407BDD6F4860B0D39BDD6F45F39F0
S123D6807FFFFFFFBDD6EACED6A2BDD71DBDCDA7BDD6F439BDD6EACED6A620EECED6587E56
S123D6A0D7043C8EFA3142652EE18FDE3D3CDE3F3C8F9641363CCC0000DD3DDD3FDD40208A
S123D6C01030A6029746EC03DD44EC05DD42BDCDA730EE00BDD71DBDCF4438C6043A3CA673
S123D6E0004326DD30C6073A3539383C3C8F3037367ED743300808BDD71D38313131316E6C
S123D70000CED63E7F0041EC02DD3FEC00052403730041973D27020D56D73E5F397F0046BB
S123D720EC02DD44EC00052403730046974227020D56D74339DC3FED02DC3D58D141465624
S123D740ED0039DC44ED02DC4258D1464656ED00397F00415F397D003E2705CC7F80DD3D1D
S123D7604F5FDD3F397D003E27037300415F39BDD71D08080808BDD704393C183CEC00BD96
S123D780D2D4183838090920AC3C183C0808BDD7040909EE00BDD11C183838EC00ED04082A
S123D7A0080808393C183CBDD704BDCECA18383824037EDE79ED00DC00ED02393C183CECA6
S123D7C002DD00EC00BDD3091838387ED7353C183CBDD704BDCE9F18383824037EDE7920D9
S123D7E05D3C183CBDD76FBDCF44183838080808087ED7353C183CBDD76FBDCF3920EBA62A
S123D800008880A700393C183CBDD76FBDCDA720093C183CBDD76FBDD04318383824037E9F
S123D820DE79080808087ED7353C183CBDD76FBDD28A183838260CCC000108080808080880
S123D840ED00390808080808086F006F01393C183CBDD76FBDD28A1838382BDB20E53C18C3
S123D8603CBDD76FBDD28A1838382ECB20D53C183CBDD76FBDD42320A13C183CBDD704BDE9
S123D880D32318383824037EDE797ED7353C183CBDD704BDD39A20EA3C183CBDD704BDD36C
S123D8A08B20DF3C183CBDD704BDD43F20D43C183CBDD704BDD42C20C93C183CBDD704BD3B
S123D8C0D4F10736BDD684320620B73C183CBDD704BDD694BDD57120A93C183CBDD704BD1C
S123D8E0D694BDD577209B3C183CBDD704BDD694BDD660208D8602E6019D47080839BDDBD3
S123D900EEA600BDDCD2A601BDDCD208082003BDDBEEA600BDDCD2A601BDDCD2080839BD10
S123D920DBEE3CEE008602E60027059D470820F738080839183CDF00BDDB4E1A83005124A7
S123D9400C8621B7C6F8DE001838180939DE00DC00C30002E300DD02830002DD04DE02EE9E
S123D960000808A60026037EDAA9812527037EDA9708A6008166261BDF02DE0409093CBD60
S123D980D704380909DF04CEC100BDD11CCEC1007EDA898164267DDF0218CEC100DE0409D7
S123D9A009DF04EC022A0C862D18A7001808CC0000A302CE000A02378FCE000A02378FCE42
S123D9C0000A02378FCE000A02378FCE000A0237183C388601335D27064FCB30E700083384
S123D9E04D27045D27064FCB30E70008334D27045D27064FCB30E70008334D27045D270645
S123DA004FCB30E7000833CB30E700085FE700CEC10020758178262ADF02DE040909DF0441
S123DA20A602BDDCB8BDDB96257217BDDB96256CA603BDDCB8BDDB96256217BDDB96255CD9
S123DA40206181632611DF02DE040909DF04A603BDDB962547204C8162261EDF02DE0409CC
S123DA6009DF04E60318CE00085886308900BDDB962529180926F2202A8173261ADF02DE56
S123DA80040909DF04EE020808A6002708BDDB96250A0820F4200CBDDB962409860ABDDB8C
S123DAA0A82006DE02087ED963DE00DC00C30002E3008FCC0000ED001838393CDC14C300D0
S123DAC0011A931426FBC30001CE0000081A931426FA8F380909ED00CC000C0909ED007EC9
S123DAE0C790090909090FDC14ED02DC120EED0039EC0008083C183CEE00AD00183838EDFB
S123DB0000390F3C183CB6103C84402605CEFF002003CEBF003CC6C03A18CEE1531AEF009C
S123DB2008083C32324D26F538CCC500EDFECCDEF3EDE2CCDEE6EDE0CE10006F226F2486C4
S123DB4030A7211C23181C22181838380E39960B84082707CC00F0DD062016DC189316235D
S123DB6007830001DD062009CC00F09316D318DD06960B84102705CC00F02012DC1A9316E9
S123DB8023058300012007CC00F09316D31A1A93062302DC06393736BDDB4E1A8300022453
S123DBA0040D323339322001370F3CDE16088CC2002603CEC110DF16A700960B84082711CA
S123DBC09C18260DDE18088CC2002603CEC110DF1838330C0E398D79CC00389D47C60C9D34
S123DBE0478D198601970F8608971C4F971DCC00019D47C6069D47C68F9D4739CC00409D47
S123DC00478602CEDC11E6009D47088CDC5126F639000A1F1F0E04000000001111110F01F9
S123DC200E00000000000C040800000F11110F010E00000C0C000C0C0000000C0C000C0413
S123DC4008020006020202120C00000A0E04000000CEDC6618CE0047A60018A700081808A6
S123DC608CDCB826F339FF0096CE10000F1D3C201D0010B700986F078104260F8601B71039
S123DC80041C0010A6031D001020228601B710041C0010A6031D0010848026EF86FFA70798
S123DCA0B60098A704E7031C00101D00101C3C20FE00960E3900000036840F8B30813A2B67
S123DCC0028B071632444444448B30813A2B028B0739BDDCB8371686029D47339D4739CEBE
S123DCE0000A02378FCE000A02378FCE000A02378FCE000A02378FCE000A02379D47CC00AD
S123DD00019D47CC00079D47CC008F9D47860233CB309D4733CB309D47C62E9D4733CB3072
S123DD209D4733CB309D4733CB309D47C66D9D47C6739D4739CC00029D478602E60027051E
S123DD409D470820F739183CDF00CC7FFFDD04CEC3001AEE0E188CC3002607CCE400DD0657
S123DD60200518EC04DD06EC0693063CDE00A300382B091A93042E04DF02DD04188CC300CF
S123DD802705183C3820CBDC041A837FFF260486012015CEC310A609814027158FC300104C
S123DDA08F8C620026F08602DE00183818097EDE793C1838DE02EE0E1AEF0CCDEF0EDE02F9
S123DDC01AEF0ECDEF0CEC0683000118ED04C30001DE00A30018ED06A60318A708EC041819
S123DDE0ED00860018A709DC0CC30001DD0C18ED0ADC00E306C30008EE068F09DF0018DF4E
S123DE000218EE0436A60018A7003209180983000126F1DE0218081AEF02DE0009DC0CED99
S123DE2000183839862020513CEC00DD00CEC300EC0A1A9300270EEE0E8CC30026F238CC69
S123DE400001ED00399C082604387ECB32183C8640A7098621B7C6F8EC0C1AEE0E8FCDEFD7
S123DE600C1AEF0E183838CC0000ED00398621B7C6F8391809860320003CDE084D260286C5
S123DE801FA70997018621B7C6F8960181202431CEDEC3A6002708BDDB9625F70820F44F75
S123DEA0D601C00A25034C20F9CB0A8B30BDDB9625FB178B30BDDB9625FB860ABDDB96254F
S123DEC0FB38390A52554E54494D45204552522000CE1000DC28E316ED161D237FB6100018
S123DEE08880B710003BCE1000DC26E31EED1E1D23F73BCE1000CC07D0E31CED1C1D23EFFE
S123DF00A622368408A7220EDE1408DF142605DE1208DF127A000A26058621B7C6F8860446
S123DF209D47848027037EE0009615843F2640960F8101223A0F4FC6CF9D47DC1E1A8300A8
S123DF40642D0BCC0000DD1E961C880C971C961C84082704C6002002C60786029D474FD6B2
S123DF6011C1102502CB30CA809D470E7EE0009639840126037EE000960F8102245EDE1A82
S123DF809C16277C088CC2002603CEC110DF1AE600960F81002634C10A26068601970F2067
S123DFA05F9611811F27594C9711811126074F37C6C09D4733C120250CC17F2208CEE060D7
S123DFC0C0203AE60086029D4720358101260DD710FCE04E9D478602970F2024810A27129C
S123DFE0CEE04ED60F3AEC009D47960F8B02970F200E8600970F86019711D610C10A26B545
S123E000D60E96398404273E96224824068B01C8102002CA10972296234824068B01C8207A
S123E0202002CA20972396244824068B01C8402002CA40972496254824068B01C88020024C
S123E040CA809725C8F0F77F0032B710223B0001000600CF020000020011495557777FFF5D
S123E060202122232425262728292A2B022D2E2F3031323334353637383904053C3D3E3F42
S123E080404142434445464748494A4B4C4D4E4F505152535455565758595A5B5C5D5E5F8C
S123E0A060616263646566036869066B6C6D6E6FF0F172737475767778017A7B7C7D7E7FAC
S123E0C018CE03E8180926FCCE10001F000433CC1BE61F00042C83000126F7203937368DE4
S123E0E056CC00029D47CEE10B8602E60027059D470820F732BDDCD232BDDCD28602C6290C
S123E1009D47CE10001C28204F06CF2A48616C7465642A2028008D1FCEE127BDDD35CE1094
S123E120001D23FB8D163B2D504F57455220474C495443482D20008601979439860E979436
S117E14039CE80004F5FE3008FC300028F8CFF0226F4393BB1
S123BFC0E153E153E153E153E153E153E153E153E153E153E153E153E153E153E153E1531D
S123BFE0DEE6DEF3E153E153E153E153E153E0C0E153E153E153E153E153E153E153C500D3
S123FFC0E153E153E153E153E153E153E153E153E153E153E153E153E153E153E153E153DD
S123FFE0DEE6DEF3E153E153E153E153E153E0C0E153E153E153E153E153E153E153C50093
S105FF020000F9
S105FF000251A8
S9030000FC
